:0200000480007A
:100000006F008004732F2034930F80006308FF0378
:10001000930F90006304FF03930FB0006300FF038E
:10002000130F000063040F0067000F00732F2034CC
:1000300063540F006F00400093E19153171F0000BD
:1000400023223FFC6FF09FFF93000000130100008C
:10005000930100001302000093020000130300004C
:100060009303000013040000930400001305000034
:10007000930500001306000093060000130700001C
:100080009307000013080000930800001309000004
:1000900093090000130A0000930A0000130B0000EC
:1000A000930B0000130C0000930C0000130D0000D4
:1000B000930D0000130E0000930E0000130F0000BC
:1000C000930F0000732540F16310050097020000B4
:1000D000938202017390523073500018970200000F
:1000E00093824202739052309B021000939252030B
:1000F0009382F2FF7390023B9302F0017390023AF5
:100100007350403097020000938242017390523046
:10011000735020307350303093010000970200007C
:10012000938282EE73905230130510001315F5017F
:10013000635C05000F00F00F930110009308D005D9
:10014000130500007300000093020000638A0200A0
:1001500073905210B7B200009B82921073902230BD
:100160007350003037250000732005307350300085
:10017000970200009382420173901234732540F17C
:1001800073002030972500009385C5E787A04500C0
:1001900027AA150003B505019B03100093931302D2
:1001A000938373009393F300938373AB9393E30070
:1001B0009383F3EE93012000631C750297250000E2
:1001C000938545E487A0050027AC150003B585019C
:1001D000B78333019B8313D09393D3009383F3B7F7
:1001E0009393730193013000631475006310300220
:1001F0000F00F00F638001009391110093E1110053
:100200009308D00513850100730000000F00F00F64
:10021000930110009308D00513050000730000003F
:10022000731000C00000000000000000000000008B
:0C023000000000000000000000000000C2
:1010000000000000000000000000000000000000E0
:1010100000000000000000000000000000000000D0
:1010200000000000000000000000000000000000C0
:1010300000000000000000000000000000000000B0
:081040000000000000000000A8
:10200000000080BF0000004000004040000080C091
:10201000EFBEADDEBEBAFECAEA1DADAB0DD03713C2
:040000058000000077
:00000001FF
